:040000000CEF00F011
:10000800FACF2FF0FBCF30F0E9CF31F083ED16F0C7
:10001800B4EF18F0700ED36E1A0EE82EFED700D08B
:10002800400E9B6E8C0E926E600E896E0F0EC16E26
:10003800F90E936E060E8A6ED80E946E3F0E8B6E76
:10004800F29ED09E000EF26E000EF16E000EF06E63
:10005800000E9E6E000EA16E000E9D6E000EA06E2C
:10006800000E9F6E000EA26E000ED76E000ED66EAA
:10007800F28AC70ED56E060E00017A6F7AC079F043
:1000880079C078F078C077F077C076F076C075F0F0
:10009800000E00016B6F000E00016A6F000E000178
:1000A8006D6F000E00016C6F12801282000E3E6EA2
:1000B8001C0E3D6EA6EC19F0216E030E216402D0D1
:1000C800000E216EF294F28E60EC18F0180E946E09
:1000D800800EC76E280EC66E000EC56E4F0EC86E17
:1000E8009E960400000ED6EC19F0D00E15EC1AF00E
:1000F800000E15EC1AF0010ED6EC19F0D10E15EC25
:100108001AF0000EB7EC19F0016E000EB7EC19F0FA
:10011800026E000EB7EC19F0036E000EB7EC19F082
:10012800046E000EB7EC19F0056E000EB7EC19F06E
:10013800066E000EB7EC19F0076E010EB7EC19F059
:10014800086E25EC1AF001380F0B070B1F6E0150D3
:100158000F0B206E02380F0B070B1D6E02500F0B92
:100168001E6E03380F0B030B1B6E03500F0B1C6E18
:1001780005380F0B030B0001806F05500F0B0001B2
:10018800816F06380F0B0001846F06500F0B0001BA
:10019800856F07380F0B0F0B0001826F07500F0B8D
:1001A8000001836F01AE26D0000ED6EC19F0D00EF8
:1001B80015EC1AF0000E15EC1AF0000E15EC1AF0FA
:1001C800000E15EC1AF0000E15EC1AF0000E15ECE6
:1001D8001AF0010E15EC1AF0010E15EC1AF0150EB6
:1001E80015EC1AF0000E15EC1AF0100E15EC1AF0BA
:1001F80025EC1AF0100E946E400EC76E200EC66ED7
:100208009E96250E0F6E030E00016E6F030E000101
:100218006F6F070E0001716F1A0E0001736F020EE7
:100228000001726F8DEC17F0700E3E6E270EC7EC52
:1002380019F0000E3E6E080E3D6EA6EC19F0296E00
:100248002950800A7F0FD8A005D02950800A670F4F
:10025800D8A00AD037EC1AF0000E3E6E080E3D6E9C
:10026800070E3F6E90EC18F0000E3E6E090E3D6EC4
:10027800A6EC19F0296E29BE05D02950800A440F32
:10028800D8A00AD037EC1AF0000E3E6E090E3D6E6B
:100298001E0E3F6E90EC18F0000E3E6E0A0E3D6E7C
:1002A800A6EC19F0296E29BE05D02950800A7E0FC8
:1002B800D8A00AD037EC1AF0000E3E6E0A0E3D6E3A
:1002C800000E3F6E90EC18F0000E3E6E0E0E3D6E66
:1002D800A6EC19F0296E29BE05D02950800A7E0F98
:1002E800D8A00AD037EC1AF0000E3E6E0E0E3D6E06
:1002F800000E3F6E90EC18F0000E3E6E100E3D6E34
:10030800A6EC19F0296E29BE05D02950800A7D0F68
:10031800D8A00AD037EC1AF0000E3E6E100E3D6ED3
:10032800000E3F6E90EC18F0000E3E6E0B0E3D6E08
:10033800A6EC19F0296E2950800A7F0FD8A005D0A5
:100348002950800A670FD8A00AD037EC1AF0000E9F
:100358003E6E0B0E3D6E140E3F6E90EC18F0000EC4
:100368003E6E0C0E3D6EA6EC19F0296E29BE05D026
:100378002950800A440FD8A00AD037EC1AF0000E92
:100388003E6E0C0E3D6E000E3F6E90EC18F0000EA7
:100398003E6E0D0E3D6EA6EC19F0296E29BE05D0F5
:1003A8002950800A7E0FD8A00AD037EC1AF0000E28
:1003B8003E6E0D0E3D6E000E3F6E90EC18F0000E76
:1003C8003E6E0F0E3D6EA6EC19F0296E29BE05D0C3
:1003D8002950800A7E0FD8A00AD037EC1AF0000EF8
:1003E8003E6E0F0E3D6E000E3F6E90EC18F0000E44
:1003F8003E6E110E3D6EA6EC19F0296E29BE05D091
:100408002950800A7D0FD8A00AD037EC1AF0000EC8
:100418003E6E110E3D6E000E3F6E90EC18F0899006
:10042800899204008AB05BD0100E946E400EC76E9D
:10043800200EC66E9E9605EC1AF0286E28BC39D0A0
:1004480047D028C0B2F00E0E0001B217D8A412D0BF
:100458000001000E3F6E00019C0E3E6E050E406EC0
:10046800610EF7EC18F0000E00016B6F000E000132
:100478006A6F129028C0B2F00E0E0001B217000188
:10048800B251020AD8A412D00001000E3F6E00013A
:10049800A10E3E6E050E406E610EF7EC18F0000ED0
:1004A80000016D6F000E00016C6F129205EC1AF0DE
:1004B800286E28C0B2F00E0E0001B2170001B2512A
:1004C8000E0AD8A4BED7400E3E6E270EC7EC19F010
:1004D80028AA05D0200E3E6E270EC7EC19F0180E7C
:1004E800946E800EC76E280EC66E000EC56E9E9660
:1004F8000400000ED6EC19F0D00E15EC1AF0000E20
:1005080015EC1AF0010ED6EC19F0D10E15EC1AF014
:10051800000EB7EC19F0016E000EB7EC19F0026E80
:10052800000EB7EC19F0036E000EB7EC19F0046E6C
:10053800000EB7EC19F0056E000EB7EC19F0066E58
:10054800000EB7EC19F0076E010EB7EC19F0086E43
:1005580025EC1AF001380F0B070B1F6E01500F0B1B
:10056800206E02380F0B070B1D6E02500F0B1E6E0C
:1005780003380F0B030B1B6E03500F0B1C6E053853
:100588000F0B030B0001806F05500F0B0001816FEB
:1005980006380F0B0001846F06500F0B0001856FA2
:1005A80007380F0B0F0B0001826F07500F0B00016C
:1005B800836F000E3E6E0A0E3D6EA6EC19F0000128
:1005C800B26F0001B205D8A464D01B500A0D1C50AC
:1005D800F326000EF422000E3E6E080E3D6EA6ECC9
:1005E80019F00001B26F0001B251F318F410D8A449
:1005F80050D01D500A0D1E50F326000EF422000E96
:100608003E6E090E3D6EA6EC19F00001B26F0001B6
:10061800B251F318F410D8A43CD0040E1F5CD8B023
:100628001AD0010E2D6E00018A6712D020A010D0BA
:10063800000E3E6E0E0E3D6EA6EC19F00001B26F74
:100648000001B205D8B48980010E00017C6F0CD07E
:100658008990000EFAD78990000E00017C6F000E79
:1006680000018A6F000E2D6E000E3E6E100E3D6E5C
:10067800A6EC19F00001B26F0001B205D8B4898266
:10068800000E3E6E100E3D6EA6EC19F0020AD8B4AC
:100698008992000E3E6E0D0E3D6EA6EC19F000011B
:1006A800B26F0001B205D8A464D01B500A0D1C50CB
:1006B800F326000EF422000E3E6E0B0E3D6EA6ECE5
:1006C80019F00001B26F0001B251F318F410D8A468
:1006D80050D01D500A0D1E50F326000EF422000EB5
:1006E8003E6E0C0E3D6EA6EC19F00001B26F0001D3
:1006F800B251F318F410D8A43CD0040E1F5CD8B043
:100708001AD0010E2E6E00018B6712D020A010D0D7
:10071800000E3E6E0F0E3D6EA6EC19F00001B26F92
:100728000001B205D8B48980020E00017C6F0CD09C
:100738008990000EFAD78990000E00017C6F000E98
:1007480000018B6F000E2E6E000E3E6E110E3D6E78
:10075800A6EC19F00001B26F0001B205D8B4898285
:10076800000E3E6E110E3D6EA6EC19F0020AD8B4CA
:100778008992040011A2F0D011B8EFD01188010EAF
:100788000001876F000E0001746F16660ED0010E0F
:10079800166E000E146E1294000E1A6E1AC019F01E
:1007A80019C018F018C017F0D8D01604D8A4D5D09E
:1007B80012B428D014660DD0000E166E1294000ED6
:1007C8001A6E1AC019F019C018F018C017F052ECB8
:1007D80019F01404D8A405D01284010E176E000E67
:1007E800186E1450020AD8A405D01284020E176E8F
:1007F800000E196E1450030AD8A4AFD01284030E49
:10080800176EA7D01704D8A444D0186619D0146658
:1008180009D01294000E176E000E1A6E1AC019F045
:1008280019C018F01404D8A403D0010E186E139040
:100838001450020AD8A42DD0020E186E000E21D032
:100848001804D8A406D013B002D0138002D0000E2A
:10085800186E1850020AD8A41CD02B6604D0000EBB
:100868002C6E010E0ED02B04D8A404D0010E2C6ED1
:10087800020E07D02B50020AD8A405D0020E2C6E07
:10088800030E2B6E06D02B50030AD8A402D0000EFC
:10089800186E1750020AD8A42DD0196623D01466F2
:1008A80009D01294000E176E000E1A6E1AC019F0B5
:1008B80019C018F01404D8A403D0010E196E1390AF
:1008C8001450020AD8A402D0020E196E1450030A5A
:1008D800D8A402D0030E196E1450040AD8A40AD062
:1008E800040E07D01904D8B413B002D0138002D074
:1008F800000E196E1750030AD8A42FD01A6623D0F9
:10090800146609D01294000E176E000E1A6E1AC0E3
:1009180019F019C018F01404D8A403D0010E1A6EE7
:1009280013901450020AD8A402D0020E1A6E145062
:10093800030AD8A402D0030E1A6E1450040AD8A4CD
:100948000CD0040E07D01A04D8B413B002D0138008
:1009580004D0000E1A6E01D01198040011A0D3D152
:1009680011B6D2D11186000E0001746F166612D02E
:10097800212A030E216402D0000E216E52EC19F0D8
:1009880037EC1AF0000E3E6E1C0E3D6E21C03FF093
:1009980090EC18F01604D8A4B7D1186609D01966D7
:1009A80007D01A6605D0140614AE02D0000E146ED5
:1009B8001804D8B404D01850020AD8A4BFD0180E0E
:1009C800946E800EC76E280EC66E000EC56E9E967B
:1009D800000ED6EC19F0D00E15EC1AF01804D8A4B5
:1009E80008D013A002D0010E01D0000E0008020F9B
:1009F800276E1850020AD8A403D02C50040F276E73
:100A0800275015EC1AF02750010D010EF324D96E6A
:100A1800000EF420DA6EDF500001B26F0F0E0001F5
:100A2800B2172750010D010EF324D96E000EF420E1
:100A3800DA6EDF500001B36F0001B3390F0B0A0DF6
:100A4800F3500001B2250001B46F0001B429276EEC
:100A580013B00AD01804D8A407D02750800A670F0B
:100A6800D8A002D0010E276E13A00AD01804D8A46B
:100A780007D02750800A440FD8A002D0000E276E56
:100A88002C660BD01850020AD8A407D02750800A29
:100A9800600FD8A002D0010E276E2C04D8A40BD06A
:100AA8001850020AD8A407D02750800A730FD8A07C
:100AB80002D0010E276E2C50020AD8A40BD0185071
:100AC800020AD8A407D02750800A1C0FD8A002D049
:100AD800000E276E2750436E446A43BE4406000E3C
:100AE800466E0A0E456E3BEC17F043C0B2F044C0A8
:100AF800B3F00001B23BF00EB2172750436E446AC0
:100B080043BE4406000E466E0A0E456E3BEC17F0D7
:100B180043500A0DF350000827240001B211276E34
:100B2800275015EC1AF025EC1AF03F0E0001B26FB1
:100B3800550EE82EFED7B22FFCD700F01904D8A422
:100B480036D013B019D0000E3E6E080E3D6EA6ECDE
:100B580019F0296E292A2950800A670FD8A002D0D7
:100B6800010E296E37EC1AF0000E3E6E080E3D6E2F
:100B780029C03FF090EC18F013A019D0000E3E6E7B
:100B8800090E3D6EA6EC19F0296E292A2950800A13
:100B9800440FD8A002D0000E296E37EC1AF0000ED0
:100BA8003E6E090E3D6E29C03FF090EC18F01950CA
:100BB800020AD8A40AD037EC1AF0000E3E6E0A0ECC
:100BC8003D6E010E3F6E90EC18F01950030AD8A440
:100BD8000AD037EC1AF0000E3E6E0E0E3D6E010E76
:100BE8003F6E90EC18F01950040AD8A419D0000EE2
:100BF8003E6E100E3D6EA6EC19F0296E292A29507A
:100C0800800A7D0FD8A002D0020E296E37EC1AF0A8
:100C1800000E3E6E100E3D6E29C03FF090EC18F0AD
:100C28001A04D8A436D013B019D0000E3E6E0B0E9D
:100C38003D6EA6EC19F0296E292A2950800A670F03
:100C4800D8A002D0010E296E37EC1AF0000E3E6EC5
:100C58000B0E3D6E29C03FF090EC18F013A019D090
:100C6800000E3E6E0C0E3D6EA6EC19F0296E292A78
:100C78002950800A440FD8A002D0000E296E37EC04
:100C88001AF0000E3E6E0C0E3D6E29C03FF090EC3F
:100C980018F01A50020AD8A40AD037EC1AF0000E3D
:100CA8003E6E0D0E3D6E010E3F6E90EC18F01A5020
:100CB800030AD8A40AD037EC1AF0000E3E6E0F0EC5
:100CC8003D6E010E3F6E90EC18F01A50040AD8A43D
:100CD8001BD0000E3E6E110E3D6EA6EC19F0296E6B
:100CE800292A2950800A7D0FD8A002D0020E296E29
:100CF80037EC1AF0000E3E6E110E3D6E29C03FF023
:100D080090EC18F001D01196040011A4EBD111BA9F
:100D1800EAD1118A000E0001746F1604D8A4CCD150
:100D280018662ED019662CD01A662AD0142A12A456
:100D380020D01704D8A407D01450800A7D0FD8A05B
:100D480002D0020E146E1750020AD8A407D014500D
:100D5800800A7B0FD8A002D0040E146E1750030A25
:100D6800D8A40ED01450800A7B0FD8A009D0040E46
:100D780006D01450800A7C0FD8A002D0030E146E3F
:100D88001804D8B404D01850020AD8A4B2D0180E47
:100D9800946E800EC76E280EC66E000EC56E9E96A7
:100DA800000ED6EC19F0D00E15EC1AF01804D8A4E1
:100DB80008D013A002D0010E01D0000E0008020FC7
:100DC800276E1850020AD8A403D02C50040F276E9F
:100DD800275015EC1AF02750010D010EF324D96E97
:100DE800000EF420DA6EDF500001B26F0F0E000122
:100DF800B2172750010D010EF324D96E000EF4200E
:100E0800DA6EDF500001B36F0001B3390F0B0A0D22
:100E1800F3500001B2250001B46F0001B405276E3C
:100E28002750800A0001B26F010E800A0001B25DEE
:100E3800D8B02BD013B005D01804D8A402D0180EFF
:100E4800276E13A006D01804D8B427AE02D03B0EE4
:100E5800276E2C6606D01850020AD8A402D01F0E9E
:100E6800276E2C04D8A406D01850020AD8A402D0A1
:100E78000C0E276E2C50020AD8A407D01850020A6C
:100E8800D8B427AE02D0630E276E2750436E446A4B
:100E980043BE4406000E466E0A0E456E3BEC17F044
:100EA80043C0B2F044C0B3F00001B23BF00EB21739
:100EB8002750436E446A43BE4406000E466E0A0E2F
:100EC800456E3BEC17F043500A0DF35000082724F9
:100ED8000001B211276E275015EC1AF025EC1AF014
:100EE8003F0E0001B26F550EE82EFED7B22FFCD789
:100EF80000F01904D8A438D013B01ED0000E3E6EEE
:100F0800080E3D6EA6EC19F0296E29062950800AB4
:100F18000001B26F010E800A0001B25DD8B002D0A4
:100F2800180E296E37EC1AF0000E3E6E080E3D6E54
:100F380029C03FF090EC18F013A016D0000E3E6EBA
:100F4800090E3D6EA6EC19F0296E290629AE02D0CD
:100F58003B0E296E37EC1AF0000E3E6E090E3D6E00
:100F680029C03FF090EC18F01950020AD8A40AD012
:100F780037EC1AF0000E3E6E0A0E3D6E000E3F6E04
:100F880090EC18F01950030AD8A40AD037EC1AF0DC
:100F9800000E3E6E0E0E3D6E000E3F6E90EC18F089
:100FA8001950040AD8A416D0000E3E6E100E3D6EDD
:100FB800A6EC19F0296E290629AE02D0000E296E7A
:100FC80037EC1AF0000E3E6E100E3D6E29C03FF051
:100FD80090EC18F01A04D8A438D013B01ED0000E24
:100FE8003E6E0B0E3D6EA6EC19F0296E29062950AF
:100FF800800A0001B26F010E800A0001B25DD8B00C
:1010080002D0180E296E37EC1AF0000E3E6E0B0E49
:101018003D6E29C03FF090EC18F013A016D0000EDA
:101028003E6E0C0E3D6EA6EC19F0296E290629AE0F
:1010380002D03B0E296E37EC1AF0000E3E6E0C0EF5
:101048003D6E29C03FF090EC18F01A50020AD8A45F
:101058000AD037EC1AF0000E3E6E0D0E3D6E000EF3
:101068003F6E90EC18F01A50030AD8A40AD037EC57
:101078001AF0000E3E6E0F0E3D6E000E3F6E90ECA5
:1010880018F01A50040AD8A42ED0000E3E6E110E85
:101098003D6EA6EC19F0296E290629AE02D0000E85
:1010A800296E37EC1AF0000E3E6E110E3D6E29C007
:1010B8003FF090EC18F017D02E6607D02D6605D0BB
:1010C8008BB402D08B8401D08B942D04D8A403D088
:1010D800010E00018A6F2E04D8A405D0010E00016C
:1010E8008B6F01D0119A1604D8B412B44BD017667E
:1010F80049D012B605D0000E146E1286129A1298B4
:10110800000E416E000EF0EC19F0BD0E476EF30EA6
:10111800466E6AEC19F0000E416E010EF0EC19F003
:10112800BE0E476EB60E466E6AEC19F0120E416E90
:10113800020EF0EC19F0BF0E476EC60E466E6AEC52
:1011480019F0120E416E030EF0EC19F0BF0E476E47
:10115800420E466E6AEC19F0120E416E040EF0EC67
:1011680019F0BF0E476EAE0E466E6AEC19F0120EFD
:10117800416E050EF0EC19F0BF0E476EBA0E466EC2
:101188006AEC19F01604D8B412A482D11704D8A4B2
:101198007FD1186646D012B605D0000E146E12869E
:1011A800129A1298000E416E000EF0EC19F0BD0E66
:1011B800476EE40E466E6AEC19F0000E416E010EA1
:1011C800F0EC19F0BE0E476EB60E466E6AEC19F0DA
:1011D800120E416E020EF0EC19F0BF0E476E7E0E35
:1011E800466E6AEC19F0120E416E030EF0EC19F01F
:1011F800BF0E476E8A0E466E6AEC19F0120E416EEB
:10120800040EF0EC19F0BF0E476E960E466E6AECAF
:1012180019F0000E416E050EF0EC19F00E0EE3EC1D
:1012280019F01804D8B404D01850020AD8A430D140
:10123800000E416E010EF0EC19F0BE0E476EB60EB0
:10124800466E6AEC19F01804D8A467D0000E416EF7
:10125800000EF0EC19F0BD0E476E990E466E6AEC62
:1012680019F0000E416E030EF0EC19F0030EE3ECDA
:1012780019F013B00BD001A004D003380F0B030BE7
:1012880008D00C0E00018C6F0C0E07D003380F0B22
:10129800010B00018C6F03500F0B00018D6F0D0EB9
:1012A80000018E6F13B001B005D00C0E00018F6FD6
:1012B8000C0E07D002380F0B0F0B00018F6F025076
:1012C8000F0B0001906F050E156E120E436E030E84
:1012D8001AEC16F0000E416E030EF0EC19F0030E36
:1012E800E3EC19F0000E416E040EF0EC19F0030E59
:1012F800E3EC19F0000E416E020EF0EC19F0BE0E90
:10130800476E200E466E6AEC19F0000E416E050E0F
:10131800F0EC19F00E0EE3EC19F01850020AD8A4FC
:10132800B7D0000E416E000EF0EC19F0BD0E476EFE
:10133800C60E466E6AEC19F0000E416E020EF0EC15
:1013480019F0BF0E476EE50E466E6AEC19F0000EF6
:10135800416E030EF0EC19F0BF0E476EE50E466EB7
:101368006AEC19F0000E416E040EF0EC19F0BF0E95
:10137800476E620E466E6AEC19F0000E416E050E5D
:10138800F0EC19F0BF0E476E620E466E6AEC19F06B
:10139800480E416E020EF0EC19F0BF0E476EE50ED6
:1013A800466E6AEC19F0480E416E030EF0EC19F027
:1013B800BF0E476EE50E466E6AEC19F0420E416E9E
:1013C800040EF0EC19F0BF0E476E620E466E6AEC22
:1013D80019F0420E416E050EF0EC19F0BF0E476E83
:1013E800620E466E6AEC19F0050E156E2C6607D073
:1013F80001B005D00C0E00018C6F0C0E07D005381B
:101408000F0B030B00018C6F05500F0B00018D6F44
:101418000B0E00018E6F2C04D8B401B005D00C0E51
:1014280000018F6F0C0E07D006380F0B010B00015F
:101438008F6F06500F0B0001906F0C0E436E020E5B
:101448001AEC16F0040E156E2C50020AD8B401B02E
:101458000BD00C0E00018C6F0C0E00018D6F0C0E62
:1014680000018E6F0C0E0DD0020E00018C6F000E65
:1014780000018D6F07380F0B0F0B00018E6F07509F
:101488000F0B00018F6F120E436E040E1AEC16F04C
:101498001604D8B412A487D01750020AD8A483D04F
:1014A800196681D012B805D0000E146E12961288F3
:1014B800129A000E416E000EF0EC19F0BE0E476E47
:1014C8003E0E466E6AEC19F0000E416E010EF0EC0D
:1014D80019F0BE0E476EB60E466E6AEC19F014503F
:1014E800800A0001B26F040E800A0001B25DD8B014
:1014F8002DD0120E416E020EF0EC19F0BF0E476EA1
:101508007E0E466E6AEC19F0120E416E030EF0EC78
:1015180019F0BF0E476E360E466E6AEC19F0120EC1
:10152800416E040EF0EC19F0BF0E476E2A0E466E9F
:101538006AEC19F0120E416E050EF0EC19F0BF0EB0
:10154800476EA20E466E6AEC19F0CFD1120E416EAC
:10155800020EF0EC19F0BF0E476E360E466E6AECBE
:1015680019F0120E416E030EF0EC19F0BF0E476E23
:101578002A0E466E6AEC19F0120E416E040EF0EC5B
:1015880019F0BF0E476EA20E466E6AEC19F0120EE5
:10159800416E050EF0EC19F0BF0E476E4E0E466E0A
:1015A8006AEC19F0A2D11604D8B412A49ED0175030
:1015B800020AD8A49AD01904D8A497D0000E416E74
:1015C800000EF0EC19F0BE0E476E5C0E466E6AEC2B
:1015D80019F0000E416E010EF0EC19F0BE0E476EC8
:1015E800B60E466E6AEC19F0000E416E020EF0EC73
:1015F80019F0BE0E476E200E466E6AEC19F0000E0A
:10160800416E030EF0EC19F0020EE3EC19F0000E37
:10161800416E040EF0EC19F0020EE3EC19F0480EDE
:10162800416E030EF0EC19F0020EE3EC19F0480ECF
:10163800416E040EF0EC19F0020EE3EC19F0000E06
:10164800416E050EF0EC19F00E0EE3EC19F0050EE4
:10165800156E000E3E6E080E3D6EA6EC19F0296E52
:1016680029504B6E4C6A4BBE4C06E1EC16F0000E4E
:10167800A4EC15F013A001B007D00C0E00018C6F7C
:101688000C0E00018D6F04D00DC08CF00EC08DF0D3
:101698000D0E00018E6F000E3E6E090E3D6EA6EC1B
:1016A80019F0296E29504B6E4C6A4BBE4C06E1EC82
:1016B80016F0000EA4EC15F013B001B007D00C0E14
:1016C80000018F6F0C0E0001906F0AD00D500C0AAC
:1016D800D8A402D0000E0D6E0DC08FF00EC090F091
:1016E8000C0E436E030E1AEC16F01604D8B412A4AE
:1016F8004ED01750020AD8A44AD01950020AD8A4CA
:1017080046D0000E416E000EF0EC19F0BE0E476E8A
:101718006B0E466E6AEC19F0000E416E010EF0EC8D
:1017280019F0BE0E476EB60E466E6AEC19F0000E42
:10173800416E020EF0EC19F0BE0E476E200E466E9A
:101748006AEC19F0000E3E6E0A0E3D6EA6EC19F01A
:10175800296E000E416E030EF0EC19F0296606D0D2
:10176800BE0E476E020E466E6AEC19F02904D8A424
:1017780006D0BE0E476E110E466E6AEC19F0000ECA
:10178800416E040EF0EC19F01C0EE3EC19F016048F
:10179800D8B412A44ED01750020AD8A44AD019506F
:1017A800030AD8A446D0000E416E000EF0EC19F0E2
:1017B800BE0E476EE30E466E6AEC19F0000E416EDF
:1017C800010EF0EC19F0BE0E476EB60E466E6AECCE
:1017D80019F0000E416E020EF0EC19F0BE0E476EC5
:1017E800200E466E6AEC19F0000E3E6E0E0E3D6E2F
:1017F800A6EC19F0296E000E416E030EF0EC19F0FC
:10180800296606D0BE0E476E020E466E6AEC19F0C7
:101818002904D8A406D0BE0E476E110E466E6AEC97
:1018280019F0000E416E040EF0EC19F01C0EE3ECFA
:1018380019F01604D8B412A458D01750020AD8A424
:1018480054D01950040AD8A450D0000E416E000E8E
:10185800F0EC19F0BE0E476ED40E466E6AEC19F025
:10186800000E416E010EF0EC19F0BE0E476EB60E7A
:10187800466E6AEC19F0000E416E020EF0EC19F09B
:10188800BE0E476E200E466E6AEC19F0000E3E6ED4
:10189800100E3D6EA6EC19F0296E000E416E030E77
:1018A800F0EC19F0296606D0BD0E476EB70E466EED
:1018B8006AEC19F02904D8A406D0BD0E476EA80E0C
:1018C800466E6AEC19F02950020AD8A406D0BD0E5B
:1018D800476ED50E466E6AEC19F0000E416E040E86
:1018E800F0EC19F01C0EE3EC19F01604D8B412A4AD
:1018F80087D01750030AD8A483D01A6681D012BAA9
:1019080005D0000E146E12961298128A000E416EBF
:10191800000EF0EC19F0BE0E476E7A0E466E6AECB9
:1019280019F0000E416E010EF0EC19F0BE0E476E74
:10193800B60E466E6AEC19F01450800A0001B26FB8
:10194800040E800A0001B25DD8B02DD0120E416E8F
:10195800020EF0EC19F0BF0E476E7E0E466E6AEC72
:1019680019F0120E416E030EF0EC19F0BF0E476E1F
:10197800360E466E6AEC19F0120E416E040EF0EC4B
:1019880019F0BF0E476E2A0E466E6AEC19F0120E59
:10199800416E050EF0EC19F0BF0E476EA20E466EB2
:1019A8006AEC19F0CFD1120E416E020EF0EC19F06C
:1019B800BF0E476E360E466E6AEC19F0120E416E77
:1019C800030EF0EC19F0BF0E476E2A0E466E6AEC55
:1019D80019F0120E416E040EF0EC19F0BF0E476EAE
:1019E800A20E466E6AEC19F0120E416E050EF0EC6E
:1019F80019F0BF0E476E4E0E466E6AEC19F0A2D172
:101A08001604D8B412A49ED01750030AD8A49AD0AA
:101A18001A04D8A497D0000E416E000EF0EC19F00D
:101A2800BE0E476EA70E466E6AEC19F0000E416EA8
:101A3800010EF0EC19F0BE0E476EB60E466E6AEC5B
:101A480019F0000E416E020EF0EC19F0BE0E476E52
:101A5800200E466E6AEC19F0000E416E030EF0EC93
:101A680019F0020EE3EC19F0000E416E040EF0ECD2
:101A780019F0020EE3EC19F0480E416E030EF0EC7B
:101A880019F0020EE3EC19F0480E416E040EF0EC6A
:101A980019F0020EE3EC19F0000E416E050EF0ECA1
:101AA80019F00E0EE3EC19F0050E156E000E3E6EE1
:101AB8000B0E3D6EA6EC19F0296E29504B6E4C6A40
:101AC8004BBE4C06E1EC16F0000EA4EC15F013A08A
:101AD80001B007D00C0E00018C6F0C0E00018D6F49
:101AE80004D00DC08CF00EC08DF00D0E00018E6F6D
:101AF800000E3E6E0C0E3D6EA6EC19F0296E2950B4
:101B08004B6E4C6A4BBE4C06E1EC16F0000EA4EC92
:101B180015F013B001B007D00C0E00018F6F0C0E3A
:101B28000001906F0AD00D500C0AD8A402D0000E04
:101B38000D6E0DC08FF00EC090F00C0E436E030EAC
:101B48001AEC16F01604D8B412A44ED01750030A93
:101B5800D8A44AD01A50020AD8A446D0000E416E22
:101B6800000EF0EC19F0BE0E476E980E466E6AEC49
:101B780019F0000E416E010EF0EC19F0BE0E476E22
:101B8800B60E466E6AEC19F0000E416E020EF0ECCD
:101B980019F0BE0E476E200E466E6AEC19F0000E64
:101BA8003E6E0D0E3D6EA6EC19F0296E000E416ECC
:101BB800030EF0EC19F0296606D0BE0E476E020E31
:101BC800466E6AEC19F02904D8A406D0BE0E476EFA
:101BD800110E466E6AEC19F0000E416E040EF0EC20
:101BE80019F01C0EE3EC19F01604D8B412A44ED068
:101BF8001750030AD8A44AD01A50030AD8A446D0CA
:101C0800000E416E000EF0EC19F0BF0E476E010E8B
:101C1800466E6AEC19F0000E416E010EF0EC19F0F8
:101C2800BE0E476EB60E466E6AEC19F0000E416E97
:101C3800020EF0EC19F0BE0E476E200E466E6AECEE
:101C480019F0000E3E6E0F0E3D6EA6EC19F0296ECF
:101C5800000E416E030EF0EC19F0296606D0BE0E98
:101C6800476E020E466E6AEC19F02904D8A406D015
:101C7800BE0E476E110E466E6AEC19F0000E416EEC
:101C8800040EF0EC19F01C0EE3EC19F01604D8B4AD
:101C980012A458D01750030AD8A454D01A50040AD2
:101CA800D8A450D0000E416E000EF0EC19F0BE0E14
:101CB800476EF20E466E6AEC19F0000E416E010E88
:101CC800F0EC19F0BE0E476EB60E466E6AEC19F0CF
:101CD800000E416E020EF0EC19F0BE0E476E200E9B
:101CE800466E6AEC19F0000E3E6E110E3D6EA6ECC3
:101CF80019F0296E000E416E030EF0EC19F02966FA
:101D080006D0BD0E476EB70E466E6AEC19F0290470
:101D1800D8A406D0BD0E476EA80E466E6AEC19F020
:101D28002950020AD8A406D0BD0E476ED50E466EBD
:101D38006AEC19F0000E416E040EF0EC19F01C0E5E
:101D4800E3EC19F01604D8A4F8D01866F6D0196692
:101D5800F4D01A66F2D0E1D0000E416E020EF0EC1B
:101D680019F0BF0E476EF30E466E6AEC19F0000EBE
:101D7800416E030EF0EC19F0BF0E476E620E466E10
:101D88006AEC19F0000E416E040EF0EC19F0BF0E6B
:101D9800476E620E466E6AEC19F0000E416E050E33
:101DA800F0EC19F0BF0E476E620E466E6AEC19F041
:101DB800C4D0000E416E020EF0EC19F0BF0E476E53
:101DC800620E466E6AEC19F0000E416E030EF0ECDE
:101DD80019F0BF0E476EF30E466E6AEC19F0000E4E
:101DE800416E040EF0EC19F0BF0E476E620E466E9F
:101DF8006AEC19F0000E416E050EF0EC19F0BF0EFA
:101E0800476E620E466E6AEC19F097D0000E416E6E
:101E1800020EF0EC19F0BF0E476E620E466E6AECC9
:101E280019F0000E416E030EF0EC19F0BF0E476E6C
:101E3800620E466E6AEC19F0000E416E040EF0EC6C
:101E480019F0BF0E476EF30E466E6AEC19F0000EDD
:101E5800416E050EF0EC19F0BF0E476E620E466E2D
:101E68006AEC19F06AD0000E416E020EF0EC19F01F
:101E7800BF0E476E620E466E6AEC19F0000E416E98
:101E8800030EF0EC19F0BF0E476E620E466E6AEC58
:101E980019F0000E416E040EF0EC19F0BF0E476EFB
:101EA800620E466E6AEC19F0000E416E050EF0ECFB
:101EB80019F0BF0E476EF30E466E6AEC19F03DD06E
:101EC800000E416E020EF0EC19F0BF0E476E620E66
:101ED800466E6AEC19F0000E416E030EF0EC19F034
:101EE800BF0E476E620E466E6AEC19F0000E416E28
:101EF800040EF0EC19F0BF0E476E620E466E6AECE7
:101F080019F0000E416E050EF0EC19F0BF0E476E89
:101F1800F30E466E6AEC19F010D01450000AD8B4CB
:101F28001BD7010AD8B445D7030AD8B46FD7010A1A
:101F3800D8B499D7070AD8B4C3D7166615EF02F0F4
:101F48002166AFD10400000E416E000EF0EC19F0CE
:101F5800BF0E476EE50E466E6AEC19F0000180511F
:101F6800300FD6EC18F000018151300FD6EC18F084
:101F78002E0ED6EC18F000018451300FD6EC18F074
:101F880000018551300FD6EC18F02E0ED6EC18F063
:101F9800BF0E476EFA0E466E6AEC19F000018251C8
:101FA800300FD6EC18F000018351300FD6EC18F042
:101FB800BF0E476EE50E466E6AEC19F0000E416ED4
:101FC800010EF0EC19F0BE0E476E210E466E6AEC5B
:101FD80019F089A207D0BF0E476EFD0E466E6AEC57
:101FE80019F006D0BF0E476EF80E466E6AEC19F06F
:101FF800000E416E020EF0EC19F089A007D0BF0E5A
:10200800476EF70E466E6AEC19F006D0BF0E476EA3
:10201800E50E466E6AEC19F0000E416E030EF0EC08
:1020280019F0BF0E476EE50E466E6AEC19F0050E04
:10203800156E1BC08CF01CC08DF020A002D00D0EB8
:1020480001D00C0E00018E6F1DC08FF01EC090F0E5
:102058000C0E436E020E1AEC16F0000E416E040EC2
:10206800F0EC19F0BE0E476E200E466E6AEC19F0C1
:10207800000E416E050EF0EC19F012A007D0BF0E4D
:10208800476EE80E466E6AEC19F079D09CC0B2F043
:10209800030E0001B217D8A452D000019DC009F068
:1020A8000A6A9EC0B5F00001B5510A26119C0AAE15
:1020B80005D0096C0A1ED8B00A2A118C09C03DF057
:1020C8000AC03EF0000E406E050E3F6E93EC19F00C
:1020D8003DC009F03EC00AF0D8900A320932D890C3
:1020E8000A320932D8900A32093211AC04D0096C8C
:1020F8000A1ED8B00A2A09C04BF00AC04CF0E1EC1D
:1021080016F0000EA4EC15F02250D6EC18F023506F
:10211800D6EC18F02450D6EC18F02450200AD8A495
:1021280004D0200ED6EC18F003D02E0ED6EC18F002
:102138002550D6EC18F0B70ED6EC18F020D09CC07D
:10214800B2F0030E0001B2170001B251010AD8A47F
:1021580006D0BF0E476EDA0E466E6AEC19F09CC0C8
:10216800B2F0030E0001B2170001B251020AD8A45E
:1021780006D0BF0E476EE10E466E6AEC19F0240ECB
:10218800416E050EF0EC19F0BF0E476EE50E466E77
:102198006AEC19F0300E416E050EF0EC19F012A23F
:1021A80007D0BF0E476EE80E466E6AEC19F079D07C
:1021B800A1C0B2F0030E0001B217D8A452D000019A
:1021C800A2C009F00A6AA3C0B6F00001B6510A26F7
:1021D800119C0AAE05D0096C0A1ED8B00A2A118CC7
:1021E80009C03DF00AC03EF0000E406E050E3F6E7D
:1021F80093EC19F03DC009F03EC00AF0D8900A32BD
:102208000932D8900A320932D8900A32093211AC10
:1022180004D0096C0A1ED8B00A2A09C04BF00AC0BB
:102228004CF0E1EC16F0000EA4EC15F02250D6ECC0
:1022380018F02350D6EC18F02450D6EC18F024509F
:10224800200AD8A404D0200ED6EC18F003D02E0E05
:10225800D6EC18F02550D6EC18F0B70ED6EC18F0DE
:1022680020D0A1C0B2F0030E0001B2170001B25194
:10227800010AD8A406D0BF0E476EDA0E466E6AEC85
:1022880019F0A1C0B2F0030E0001B2170001B2515B
:10229800020AD8A406D0BF0E476EE10E466E6AEC5D
:1022A80019F02104D8A49FD1010E156E010E00016A
:1022B8008C6F000E436E000E1AEC15F0100E416E76
:1022C800000EF0EC19F0000E31EC1AF0000E31ECB3
:1022D8001AF0100E416E010EF0EC19F0000E31EC00
:1022E8001AF0000E31EC1AF012A017D0120E416E3F
:1022F800000EF0EC19F0BF0E476E720E466E6AECD7
:1023080019F0120E416E010EF0EC19F0BF0E476E77
:10231800660E466E6AEC19F08ED09CC0B2F0030EC1
:102328000001B217D8A45AD000019DC009F00A6A6A
:102338009EC0B7F00001B7510A26119C0AAE05D01D
:10234800096C0A1ED8B00A2A118C09C03DF00AC0CF
:102358003EF0000E406E050E3F6E93EC19F03DC046
:1023680009F03EC00AF0D8900A320932D8900A32F1
:102378000932D8900A32093211AC04D0096C0A1E0D
:10238800D8B00A2A09C04BF00AC04CF0E1EC16F0AC
:10239800010EA4EC15F0050E156E0BC08CF00CC0E8
:1023A8008DF00DC08EF00B0E00018F6F0EC090F0F7
:1023B800120E436E000E1AEC16F04E0E416E000E11
:1023C800F0EC19F0B70ED6EC18F04E0E416E010E77
:1023D800F0EC19F0200ED6EC18F02DD0120E416E4C
:1023E800000EF0EC19F00B0EE3EC19F0120E416E32
:1023F800010EF0EC19F09CC0B2F0030E0001B21708
:102408000001B251010AD8A406D0BF0E476E5A0E79
:10241800466E6AEC19F09CC0B2F0030E0001B217C8
:102428000001B251020AD8A406D0BF0E476E1E0E94
:10243800466E6AEC19F0000E416E020EF0EC19F0CF
:10244800BE0E476EC50E466E6AEC19F0BE0E476E9C
:10245800200E466E6AEC19F0010E156E020E000190
:102468008C6F000E436E040E1AEC15F0100E416EC0
:10247800040EF0EC19F0000E31EC1AF0000E31ECFD
:102488001AF0100E416E050EF0EC19F0000E31EC4A
:102498001AF0000E31EC1AF012A217D0120E416E8B
:1024A800040EF0EC19F0BF0E476E720E466E6AEC21
:1024B80019F0120E416E050EF0EC19F0BF0E476EC2
:1024C800660E466E6AEC19F08ED0A1C0B2F0030E0B
:1024D8000001B217D8A45AD00001A2C009F00A6AB4
:1024E800A3C0B8F00001B8510A26119C0AAE05D065
:1024F800096C0A1ED8B00A2A118C09C03DF00AC01E
:102508003EF0000E406E050E3F6E93EC19F03DC094
:1025180009F03EC00AF0D8900A320932D8900A323F
:102528000932D8900A32093211AC04D0096C0A1E5B
:10253800D8B00A2A09C04BF00AC04CF0E1EC16F0FA
:10254800010EA4EC15F0050E156E0BC08CF00CC036
:102558008DF00DC08EF00B0E00018F6F0EC090F045
:10256800120E436E040E1AEC16F04E0E416E040E57
:10257800F0EC19F0B70ED6EC18F04E0E416E050EC1
:10258800F0EC19F0200ED6EC18F02DD0120E416E9A
:10259800040EF0EC19F00B0EE3EC19F0120E416E7C
:1025A800050EF0EC19F0A1C0B2F0030E0001B2174D
:1025B8000001B251010AD8A406D0BF0E476E5A0EC8
:1025C800466E6AEC19F0A1C0B2F0030E0001B21712
:1025D8000001B251020AD8A406D0BF0E476E1E0EE3
:1025E800466E6AEC19F02150020AD8A40DD1000EEB
:1025F800416E000EF0EC19F0BE0E476E4D0E466EA1
:102608006AEC19F0BE0E476EB60E466E6AEC19F00B
:1026180012A012D0000E416E020EF0EC19F00E0E50
:10262800E3EC19F0BE0E476E2F0E466E6AEC19F0F9
:102638001C0EE3EC19F0E8D09CC0B2F0030E0001C8
:10264800B217D8A463D000019DC009F00A6A9EC0E1
:10265800B9F00001B9510A26119C0AAE05D0096CDF
:102668000A1ED8B00A2A118C09C03DF00AC03EF0F3
:10267800000E406E050E3F6E93EC19F03DC009F058
:102688003EC00AF0D8900A320932D8900A3209328C
:10269800D8900A32093211AC04D0096C0A1ED8B09D
:1026A8000A2A09C04BF00AC04CF0E1EC16F0010E02
:1026B800A4EC15F0050E156E0BC08CF00CC08DF057
:1026C8000DC08EF00B0E00018F6F0EC090F0000E43
:1026D800436E020E1AEC16F03C0E416E020EF0EC40
:1026E80019F0B70ED6EC18F0BF0E476EEF0E466E17
:1026F8006AEC19F03C0E416E030EF0EC19F0BF0EB7
:10270800476E180E466E6AEC19F028D0000E416E1E
:10271800020EF0EC19F00E0EE3EC19F09CC0B2F0CA
:10272800030E0001B2170001B251010AD8A406D065
:10273800BF0E476E100E466E6AEC19F09CC0B2F0E0
:10274800030E0001B2170001B251020AD8A406D044
:10275800BF0E476E1D0E466E6AEC19F0000E416EF4
:10276800040EF0EC19F0BE0E476EB60E466E6AEC1B
:1027780019F00001A0510001BC6F0001BB6B000102
:102788009F510001BB250001BB6F000E0001BC2159
:102798000001BC6FBBC043F0BCC044F0000E466EE5
:1027A800050E456E3BEC17F043C0BBF044C0BCF0CF
:1027B800D8900001BB350001BB6F0001BC3500019A
:1027C800BC6FBBC04BF0BCC04CF0E1EC16F0000E87
:1027D800A4EC15F0000E416E050EF0EC19F0BF0EDA
:1027E800476ED00E466E6AEC19F02350D6EC18F0FE
:1027F8002C0ED6EC18F02450D6EC18F02550D6EC58
:1028080018F0760ED6EC18F02150030AD8A415EF6C
:1028180002F0000E416E000EF0EC19F0BE0E476E8D
:10282800890E466E6AEC19F0BE0E476EB60E466EFD
:102838006AEC19F012A213D0000E416E020EF0ECF1
:1028480019F00E0EE3EC19F0BE0E476E2F0E466E11
:102858006AEC19F01C0EE3EC19F015EF02F0A1C0B8
:10286800B2F0030E0001B217D8A460D00001A2C0D4
:1028780009F00A6AA3C0BAF00001BA510A26119CED
:102888000AAE05D0096C0A1ED8B00A2A118C09C0F4
:102898003DF00AC03EF0000E406E050E3F6E93EC10
:1028A80019F03DC009F03EC00AF0D8900A3209324A
:1028B800D8900A320932D8900A32093211AC04D0C1
:1028C800096C0A1ED8B00A2A09C04BF00AC04CF09D
:1028D800E1EC16F0010EA4EC15F0050E156E0BC018
:1028E8008CF00CC08DF00DC08EF00B0E00018F6FB8
:1028F8000EC090F0000E436E020E1AEC16F03C0E5D
:10290800416E020EF0EC19F0B70ED6EC18F0BF0EBF
:10291800476EEF0E466E6AEC19F03C0E416E030EE0
:10292800F0EC19F0040EE3EC19F028D0000E416E1B
:10293800020EF0EC19F00E0EE3EC19F0A1C0B2F0A3
:10294800030E0001B2170001B251010AD8A406D043
:10295800BF0E476E100E466E6AEC19F0A1C0B2F0B9
:10296800030E0001B2170001B251020AD8A406D022
:10297800BF0E476E1D0E466E6AEC19F0000E416ED2
:10298800040EF0EC19F0BE0E476EB60E466E6AECF9
:1029980019F00001A5510001BE6F0001BD6B0001D7
:1029A800A4510001BD250001BD6F000E0001BE212C
:1029B8000001BE6FBDC043F0BEC044F0000E466EBD
:1029C800050E456E3BEC17F043C0BDF044C0BEF0A9
:1029D800D8900001BD350001BD6F0001BE35000172
:1029E800BE6FBDC04BF0BEC04CF0E1EC16F0000E5F
:1029F800A4EC15F0000E416E050EF0EC19F0BF0EB8
:102A0800476ED00E466E6AEC19F02350D6EC18F0DB
:102A18002C0ED6EC18F02450D6EC18F02550D6EC35
:102A280018F0760ED6EC18F015EF02F00001B16F31
:102A3800000E0001AA6F0001B1290001A66F000174
:102A4800000E0001AE6F00018C0E0001AD6F43C097
:102A580041F00001B151F0EC19F0000115C0A7F0E8
:102A68000001A86B5CD0ADC0D9FFAEC0DAFFDF5063
:102A7800446E44AE03D00001A96903D0000E0001E2
:102A8800A96FADC0D9FFAEC0DAFFDF50446E1F0E8C
:102A9800441644500001AF6F0001B06B0001AA5109
:102AA800100D0001AFC044F00001B0C045F0050EA4
:102AB800D89044364536E82EFBD7F350442400011D
:102AC800AF6FF45045200001B06F000E0001AC6FED
:102AD800000E0001AB6F100E0001AB5D000E00018F
:102AE800AC59D8B015D0390E0001AF25F66EBD0E21
:102AF8000001B021F76E0800F5500001A91931EC6A
:102B08001AF00001AF4BB02B0001AB4BAC2BE3D755
:102B18000001A707D8A0A8070001AD4BAE2B000104
:102B2800A851A711D8A49FD70001A6510001B163ED
:102B380001D005D00001B12B0001AA2B80D71200CB
:102B48002A6606D0200E2A6E266602D0200E266E31
:102B5800000150A010D02650200AD8B403D02D0E62
:102B68002A6E09D01050200AD8B403D02D0E266E34
:102B780002D02D0E106E2A50200AD8B40AD02A503E
:102B88002D0AD8B406D02A50300F226E2AC00BF076
:102B98000ED02AC022F02A50200AD8A402D00C0E47
:102BA8000B6E2A502D0AD8A402D00A0E0B6E26509E
:102BB800200AD8B40AD026502D0AD8B406D02650F8
:102BC800300F236E26C00CF00ED026C023F02650FE
:102BD800200AD8A402D00C0E0C6E26502D0AD8A4B8
:102BE80002D00A0E0C6E1050200AD8B40AD0105029
:102BF8002D0AD8B406D01050300F246E10C00DF036
:102C08000ED010C024F01050200AD8A402D00C0E08
:102C18000D6E10502D0AD8A402D00A0E0D6E7BC07E
:102C28000EF000017B51300F256E12004F6E4F28B9
:102C38004E6E0001000E4B6E00018C0E4A6E43C0B2
:102C480041F04F50F0EC19F015C045F0466A4BD0F2
:102C58004AC0D9FF4BC0DAFFDF50446E44AE02D001
:102C6800476802D0000E476E4AC0D9FF4BC0DAFF52
:102C7800DF50446E1F0E441644504C6E4D6A4CC0D3
:102C88003DF04DC03EF0000E406E180E3F6E93ECC6
:102C980019F03DC04CF03EC04DF04E504F6204D08C
:102CA8000C0E4C26000E4D22000E496E000E486E8A
:102CB8000C0E485C000E4958D8B010D0E90E4C24D0
:102CC800F66EBB0E4D20F76E0800F550471831EC34
:102CD8001AF04C4A4D2A484A492AEAD74506D8A04C
:102CE80046064A4A4B2A46504510D8A4B1D74E50FA
:102CF8004F6201D003D04EC04FF09BD712000600A0
:102D0800EACF32F0E1CF33F0E2CF34F0D9CF35F06B
:102D1800DACF36F0F3CF37F0F4CF38F0F6CF39F01A
:102D2800F7CF3AF0F8CF3BF0F5CF3CF0F2BAF2A487
:102D380027D0F29420EC18F000016A4B6B2B0001AD
:102D48006C4B6D2B00016B514E0A200ED8B46A19DA
:102D5800D8A407D01280000E00016B6F000E00018E
:102D68006A6F00016D514E0A200ED8B46C19D8A4B0
:102D780007D01282000E00016D6F000E00016C6F0B
:102D88003CC0F5FF3BC0F8FF3AC0F7FF39C0F6FF7B
:102D980038C0F4FF37C0F3FF36C0DAFF35C0D9FFBB
:102DA80034C0E2FF33C0E1FF32C0EAFF31C0E9FFBF
:102DB80030C0FBFF2FC0FAFF1100000150904CAE4D
:102DC80006D04B1E4C1E4B4A4C2A00015080270E41
:102DD800406E100E3F6E4BC03DF04CC03EF0D8EC3C
:102DE80017F03DC043F03EC044F0030E466EE80EB7
:102DF800456E3BEC17F043502A6E030E406EE80E0A
:102E08003F6E4BC03DF04CC03EF0D8EC17F03DC0D3
:102E180043F03EC044F0000E466E640E456E3BEC37
:102E280017F04350266E000E406E640E3F6E4BC086
:102E38003DF04CC03EF0D8EC17F03DC043F03EC02A
:102E480044F0000E466E0A0E456E3BEC17F04350F8
:102E5800106E4BC03DF04CC03EF0000E406E0A0EA6
:102E68003F6ED8EC17F03D5000017B6F1200000E4A
:102E7800486E4650800AF36E800EF35C000ED8B49C
:102E8800455CD8B006D0456C461ED8B0462A010E1F
:102E9800486E4450800AF36E800EF35C000ED8B47E
:102EA800435CD8B006D0436C441ED8B0442A010E07
:102EB800481A000E4A6E000E496E46504510D8B4A6
:102EC8001CD0010E476E04D0D89045364636472AA6
:102ED80046AEFAD7D89049364A364550435C4650F4
:102EE8004458D8A005D04550435E4650445A4980BE
:102EF800D89046324532472EEDD74850D8B404D042
:102F0800496C4A1ED8B04A2A49C043F04AC044F026
:102F180012008A940001000E3F6E0001C40E3E6E3E
:102F2800050E406E2A0E35EC19F00001000E3F6EBA
:102F38000001BF0E3E6E050E406E2B0E35EC19F0EB
:102F4800050E3E6E310EC7EC19F0050E3E6E320EC0
:102F5800C7EC19F06EC03EF0210EC7EC19F06FC037
:102F68003EF0220EC7EC19F00FC03EF0250EC7EC5C
:102F780019F071C03EF0260EC7EC19F072C03EF091
:102F8800230EC7EC19F0010E3E6E3C0EC7EC19F08B
:102F9800060E3E6E3D0EC7EC19F00F0E3E6E200E6B
:102FA800C7EC19F08A841200000E426E3E50800A67
:102FB800F36E800EF35C000ED8B43D5CD8B006D03A
:102FC8003D6C3E1ED8B03E2A010E426E4050800A2B
:102FD800F36E800EF35C000ED8B43F5CD8B004D01A
:102FE8003F6C401ED8B0402A40503F10D8B418D08B
:102FF800010E416E04D0D8903F364036412A40AE8B
:10300800FAD73F503D5C40503E58D8A004D03F50BE
:103018003D5E40503E5AD89040323F32412EF1D763
:103028004250D8B404D03D6C3E1ED8B03E2A3DC0B4
:103038003DF03EC03EF0120081B60AD011B011D06A
:10304800060E0001756F0001762F0BD0118009D094
:1030580011A007D0060E0001766F0001752F01D070
:10306800119081B80AD011B211D0060E0001776F05
:103078000001782F0BD0118209D011A207D0060EBB
:103088000001786F0001772F01D0119281BA0AD020
:1030980011B411D0060E0001796F00017A2F0BD000
:1030A800118409D011A407D0060E00017A6F00011F
:1030B800792F01D01194120004008B948B828B809D
:1030C80000D000D08B927FEC19F07FEC19F08B8246
:1030D8007FEC19F07FEC19F0210E2BEC1AF0C20EE0
:1030E8002BEC1AF0070E2BEC1AF0130E2BEC1AF03F
:1030F800200E2BEC1AF0090E2BEC1AF052EC19F0FA
:10310800080E2BEC1AF00C0E2BEC1AF0000E416E88
:10311800000EF0EC19F01200000E436E3EC040F0B5
:1031280040C041F0426A4150030BAA6E3DC0A9FF5E
:103138003FC0A8FFA69EA69CA684000EF2BE010E64
:10314800436EF29E550EA76EAA0EA76EA682A6B271
:10315800FED743B002D0F29E01D0F28EA6941200A0
:1031680000EE60F0460EEE6AE806FDE1506A00EEF9
:1031780001F02E0EEE6AE806FDE13A0EF66E340E08
:10318800F76E000EF86E00EEBFF010EE0FF00900BB
:10319800F5CFEEFFE550E150FAE1000EF86E0001C0
:1031A8000EEF00F0416E4150060DF3CF42F0F4CF20
:1031B80043F0000E456E000E446E060E445C000E91
:1031C8004558D8B00FD0C10E4224F66EB10E432038
:1031D800F76E0800F55031EC1AF0424A432A444A87
:1031E800452AEBD71200426E8A9242500DEC1AF033
:1031F800416E020EE82EFED700D0000E436E0DD0B1
:103208004350010DF3503E24D96EF4503F20DA6E3E
:10321800000E0DEC1AF0DF6E432A4050435CD8A034
:10322800EFD78A8212003E6E040089988B90000EB8
:103238003F6E12D03E50800B3D6E3D6602D0899A9B
:1032480001D0898A00D000D0898800D000D0899820
:103258003E503E243E6E3F2A070E3F64EBD78B80DC
:103268001200426E8A9242500DEC1AF0416E020E24
:10327800E82EFED700D0000E436E0AD03EC0D9FF1C
:103288003FC0DAFFDF500DEC1AF03E4A3F2A432ACE
:103298004050435CD8A0F2D78A821200000E416EDB
:1032A800000EF0EC19F0000E446E000E436E445010
:1032B800800A7F0FF80ED8B4435CD8B006D0000E51
:1032C80031EC1AF0434A442AF2D712000AD046C019
:1032D800F6FF47C0F7FF0800F550D6EC18F0464A4D
:1032E800472A46C0F6FF47C0F7FF0800F550000917
:1032F800D8B41200ECD7000E3E6E0DD0000E3D6E15
:1033080006D00400530EE82EFED700F03D2AC70E63
:103318003D64F7D73E2A010E3E64F0D712003D50B7
:103328003F02F3CF41F0F4CF42F03D504002F3505A
:1033380042263E503F02F350422641C03DF042C073
:103348003EF012003EC03FF03FC040F0416A40509E
:10335800030BAA6E3DC0A9FFA69CA69EA68000F0FE
:1033680000F0A85012003E6EFCEC19F0C586C7A00C
:10337800FED73EB002D0C59A01D0C58AC588C5B867
:10338800FED7C9501200406E8A9240500DEC1AF0D8
:103398003F6E3E500DEC1AF08A820A0EE82EFED7D8
:1033A80000D012003E6EFCEC19F03E6604D0C580D9
:1033B800C5A004D0FDD7C582C5B2FED71200466E9F
:1033C800000E476E04D0200ED6EC18F0472A46505F
:1033D800475CD8B01200F7D7426E4250070B40093D
:1033E8002BEC1AF041507F0B80092BEC1AF01200DD
:1033F8000400C5CF3DF01F0E3D16D8B4C7B4F9D7A9
:1034080012008A92FF0E0DEC1AF03E6E8A823E5030
:1034180012003D6E3DC0C9FF9EA6FED79E96C950BC
:1034280012003E6EFCEC19F03EC0C9FFC7A01200A6
:10343800FDD732ECEEC40031ECEEC40031ECEEC442
:103448000000FCEC19F0C584C5A41200FDD7406E3D
:10345800899C405017EC19F01200406E898C40503E
:0C34680017EC19F01200A6A21200FDD70C
:10B1C00000000000000000003E4551453E003E6B7F
:10B1D0006F6B3E001C3E7C3E1C00183C7E3C180001
:10B1E00030367F363000185C7E5C1800001818007E
:10B1F00000FFFFE7E7FFFF003C24243C00FFC3DB28
:10B20000DBC3FF0030484A360E00062979290600C4
:10B2100060703F020400607E0A353F002A1C361C25
:10B220002A00007F3E1C0800081C3E7F00001436E8
:10B230007F361400005F005F000006097F017F0079
:10B24000224D5559220060606060000014B6FFB6C0
:10B25000140004067F06040010307F301000080838
:10B260003E1C0800081C3E08080078404040400092
:10B27000083E083E0800303C3F3C3000030F3F0FC3
:10B28000030000000000000000065F060000070346
:10B2900000070300247E247E2400242B6A12000071
:10B2A000631308646300364956205000000703000A
:10B2B0000000003E4100000000413E000000083E4A
:10B2C0001C3E080008083E08080000E0600000007E
:10B2D000080808080800006060000000201008044A
:10B2E00002003E4141413E0000427F400000625169
:10B2F000494946002249494936001814127F100076
:10B300002F49494931003C4A49493000017109053A
:10B310000300364949493600064949291E00006C98
:10B320006C00000000EC6C000000081422410000DA
:10B330002424242424000041221408000201590975
:10B3400006003E415D551E007E1111117E007F49B1
:10B35000494936003E41414122007F4141413E0082
:10B360007F49494941007F09090901003E41494996
:10B370007A007F0808087F0000417F4100003040CC
:10B3800040403F007F08142241007F404040400081
:10B390007F0204027F007F0204087F003E4141419A
:10B3A0003E007F09090906003E4151215E007F09E8
:10B3B0000919660026494949320001017F0101004F
:10B3C0003F4040403F001F2040201F003F403C4086
:10B3D0003F006314081463000708700807007149F0
:10B3E00045430000007F4141000002040810200096
:10B3F0000041417F000004020102048080808080BF
:10B4000080000003070000002054545478007F445B
:10B4100044443800384444442800384444447F00BD
:10B42000385454540800087E0909000018A4A4A444
:10B430007C007F040478000000007D400000408014
:10B44000847D00007F102844000000007F40000041
:10B450007C04180478007C040478000038444444D8
:10B460003800FC444444380038444444FC004478E8
:10B4700044040800085454542000043E44240000AE
:10B480003C40207C00001C2040201C003C603060C0
:10B490003C006C10106C00009CA0603C00006454E8
:10B4A000544C0000083E41410000000077000000BD
:10B4B0000041413E08000201020100003C26232613
:10B4C0003C441144114411AA55AA55AA55BBEEBBE0
:10B4D000EEBBEE000000FF0000080808FF00000AB5
:10B4E0000A0AFF000008FF00FF000008F808F80043
:10B4F000000A0A0AFE00000AFB00FF000000FF002D
:10B50000FF00000AFA02FE00000A0B080F00000804
:10B510000F080F00000A0A0A0F0000080808F800C8
:10B52000000000000F08080808080F0808080808AD
:10B53000F80808000000FF080808080808080808BC
:10B540000808FF0808000000FF0A0A00FF00FF08C3
:10B5500008000F080B0A0A00FE02FA0A0A0A0B0882
:10B560000B0A0A0AFA02FA0A0A00FF00FB0A0A0A90
:10B570000A0A0A0A0A0AFB00FB0A0A0A0A0A0B0A52
:10B580000A080F080F08080A0A0AFA0A0A08F8083F
:10B59000F80808000F080F08080000000F0A0A004A
:10B5A0000000FE0A0A00F808F8080808FF08FF086B
:10B5B00008007E4B4A4B420A0A0AFF0A0A0808089A
:10B5C0000F0000000000F80808FFFFFFFFFFFFF07A
:10B5D000F0F0F0F0F0FFFFFF000000000000FFFFC0
:10B5E000FF0F0F0F0F0F0F003E4949412200385443
:10B5F0005444280001407E40010000017C410000CD
:10B6000027484B483F009DA2623D000006090906FD
:10B6100000003855545508000018180000000008B4
:10B620000000000030403E02027F06187F13132AFC
:10B630003E14143E2A003C3C3C3C0000000000004C
:10B6400000007E1111117E007F49494931007F4978
:10B65000494936007F01010101C07E41417FC000A0
:10B660007F494949410077087F087722494949368F
:10B6700000007F2010087F007E2111097E007F08D6
:10B6800014224100407E01017F007F0204027F00FE
:10B690007F0808087F003E4141413E007F010101D3
:10B6A0007F007F09090906003E4141412200010156
:10B6B0007F010100274848483F000E117F110E000E
:10B6C0006314081463007F40407FC0000708080827
:10B6D0007F007F407F407F007F407F40FF03017FEE
:10B6E000484830007F4848307F007F484848300055
:10B6F000224149493E007F083E413E006619090942
:10B700007F002054545478003C4A4A4A31007C540B
:10B71000545428007C04040C00C07844447CC000CD
:10B720003854545408006C107C106C002844545455
:10B7300028007C2010087C007C20120A7C007C10F1
:10B74000284400403804047C00007C0810087C0079
:10B750007C1010107C003844444438007C040404FD
:10B760007C00FC4444443800384444442800040429
:10B770007C0404009CA0603C000018247C24180079
:10B780006C10106C00007C40407CC0000C1010104D
:10B790007C007C407C407C007C407C40FC0C047C39
:10B7A000505020007C5050207C007C505050200095
:10B7B0002844545438007C10384438004834141459
:10B7C0007CE0F0F8F4EE1F1F1F1F1F1F1F1FEEF479
:10B7D000F8F0E0001F3F7F3F1F0000000000000066
:10B7E000001F3F7F3F1F00FCFEFFFEFC000000002B
:10B7F00000000000FCFEFFFEFC0003070F173B7C6F
:10B800007C7C7C7C7C7C7C3B170F07030000000069
:10B8100000000000F0F8FCF8F0000000000000005C
:10B82000000000000000001F3F7F3F1F00000000DD
:10B8300000000000000000000000FCFEFFFEFC0015
:10B8400000000000000000000000000000070F1FC3
:10B850000F0700000000000000000000040E1F1F82
:10B860001F1F1F1F1F1FEEF4F8F0E00000000080F4
:10B87000C0E0E0E0E0E0E0E0E0DFBF7F3F1F00FC91
:10B88000FEFFFEFD030303030303030301000000A7
:10B89000000003070F173B7C7C7C7C7C7C7C7C3825
:10B8A0001000000000000000040E1F1F1F1F1F1FBC
:10B8B0001F1FEEF4F8F0E00000000080C0E0E0E0C0
:10B8C000E0E0E0E0E0DFBF7F3F1F0000000000019C
:10B8D0000303030303030303FDFEFFFEFC0000005C
:10B8E0000010387C7C7C7C7C7C7C7C3B170F0703C5
:10B8F00000F0F8FCF8F00000000000000000F0F894
:10B90000FCF8F0001F3F7FBFDFE0E0E0E0E0E0E0B8
:10B91000E0DFBF7F3F1F00000000000103030303BF
:10B9200003030303FDFEFFFEFC0000000000000017
:10B9300000000000000000070F1F0F0700E0F0F8F4
:10B94000F4EE1F1F1F1F1F1F1F1F0E04000000000B
:10B950001F3F7FBFDFE0E0E0E0E0E0E0E0C080002C
:10B9600000000000000000010303030303030303BE
:10B97000FDFEFFFEFC0000000010387C7C7C7C7C1F
:10B980007C7C7C3B170F070300E0F0F8F4EE1F1FF0
:10B990001F1F1F1F1F1F0E04000000001F3F7FBF3F
:10B9A000DFE0E0E0E0E0E0E0E0C08000000000FC7C
:10B9B000FEFFFEFD0303030303030303FDFEFFFE7F
:10B9C000FC0003070F173B7C7C7C7C7C7C7C7C3BF5
:10B9D000170F070300000000040E1F1F1F1F1F1F6B
:10B9E0001F1FEEF4F8F0E00000000000000000006F
:10B9F00000000000001F3F7F3F1F0000000000000C
:10BA00000000000000000000FCFEFFFEFC00000043
:10BA10000000000000000000000000070F1F0F07DB
:10BA200000E0F0F8F4EE1F1F1F1F1F1F1F1FEEF492
:10BA3000F8F0E0001F3F7FBFDFE0E0E0E0E0E0E0A3
:10BA4000E0DFBF7F3F1F00FCFEFFFEFD030303039B
:10BA500003030303FDFEFFFEFC0003070F173B7CFF
:10BA60007C7C7C7C7C7C7C3B170F070300E0F0F83F
:10BA7000F4EE1F1F1F1F1F1F1F1FEEF4F8F0E00042
:10BA80001F3F7FBFDFE0E0E0E0E0E0E0E0DFBF7F1E
:10BA90003F1F00000000000103030303030303032F
:10BAA000FDFEFFFEFC0000000010387C7C7C7C7CEE
:10BAB0007C7C7C3B170F07030000000000000000A7
:10BAC0000000000000000000000000000000000076
:10BAD0000080C0C0C0C0C0C0C0C080000000000066
:10BAE000000000000103030303030303030100003C
:10BAF0000000000000000000000000000000000046
:10BB00000000000000000000000000000000000035
:10BB10000000000000000000000000000000000025
:10BB20000000000000000000000000000000000015
:10BB30000000000000000000000000000000000005
:10BB40000000000000F0F0F0F00000000000000035
:10BB500000000000000000000000000000000000E5
:10BB600000000000000000000000000000000000D5
:10BB700000000000000000000000000000000000C5
:10BB800000000000000000000000000000000000B5
:10BB900000000000000000000000000000000000A5
:10BBA0000000000000000000000000000000000095
:10BBB000000000000000000F0F0F0F000000000049
:10BBC00000000000000000000000F0F0F0F00000B5
:10BBD0000000000000000000000000000000000065
:10BBE00000000000000000000000F8FE060383C310
:10BBF00063331EFEF800071F1E3331303030181F2C
:10BC0000070000000C0C0EFFFF0000000000000009
:10BC10003030303F3F30303000001C1E07030383BC
:10BC2000C3E3773E1C0030383C3E37333130303090
:10BC300030000C0E07C3C3C3C3C3E77E3C000C1C1B
:10BC4000383030303030391F0E00C0E070381C0EF4
:10BC500007FFFF000000030303030303033F3F0349
:10BC600003003F7F636363636363E3C383000C1C70
:10BC7000383030303030381F0F00C0F0F8DCCEC71D
:10BC8000C3C3C38000000F1F393030303030391F3C
:10BC90000F00030303030303C3F33F0F030000007C
:10BCA00000303C0F03000000000000BCFEE7C3C3EF
:10BCB000C3E7FEBC00000F1F393030303030391F71
:10BCC0000F003C7EE7C3C3C3C3C3E7FEFC00000014
:10BCD000303030381C0E0703000080808080808068
:10BCE000808080800000010101010101010101014A
:10BCF0000000000000000000000000000000000044
:10BD0000003838380000000000000000000000008B
:10BD10000000000000000000000000000000000023
:10BD20000000000000001C1C1C00000000000000BF
:10BD300000001C1C1C00000000FC068309012141BE
:10BD400086412111098306FC001F306048404040B5
:10BD5000604040404860301F000000FFE1FF00AA43
:10BD6000AAAA000080C00000000C1E3F3F3F1E0C2E
:10BD700000000001001F0000000000FFE1FF00AA1A
:10BD8000AAAA008040408000000C1E3F3F3F1E0CCE
:10BD9000000000181412110000D3F1F2E0ED2E2083
:10BDA000E2F0E5ECE5EDE800D3EFF02EE2EAEBFEA1
:10BDB000F7E5EDE8E5EC00D0E5EBE520EEF2EAEBA7
:10BDC000FEF7E5EDEE00D3F1F2E0EDEEE2EAE02081
:10BDD000E4E0F2FB00D3EFF02EEEF2EAEB2DEDE81B
:10BDE000E5EC20002020C2F0E5ECFF2FC4E0F2E0FB
:10BDF0002020002020CDE0F1F2F0EEE9EAE820205A
:10BE00002000202020CEF2EAEBFEF7E5ED202020F6
:10BE100000202020C2EAEBFEF7E5ED2020202000E4
:10BE20002020202020202020202020202020002032
:10BE300020CDC5D220D1C2DFC7C8212020002020BC
:10BE4000C1F3E4E8EBFCEDE8EA20312000D0E0E4C7
:10BE5000E8EEE4E0F2F7E8EA20312000C2F0E5EC99
:10BE6000FF20E1F3E4E8EB2E312000D0E5E6E8EC3A
:10BE700020E1F3E4F3EB2E3120002020C1F3E4E8CD
:10BE8000EBFCEDE8EA20322000D0E0E4E8EEE4E06C
:10BE9000F2F7E8EA20322000D0E5E6E8EC20E1F312
:10BEA000E4E8EB2E322000C2F0E5ECFF20E1F3E401
:10BEB000E8EB2E3220002D2D2D2D2D2D2D2D2D2D6D
:10BEC0002D2D2D2D002E2E2E2E2E2E2E2E2E2E2EC4
:10BED0002E2E2E00D3EFF02EF0E5EBE520E1F3E47B
:10BEE0002E3100C7F3ECECE5F020E1F3E4E8EB2EB3
:10BEF0003100D3EFF02EF0E5EBE520E1F3E42E3254
:10BF000000C7F3ECECE5F020E1F3E4E8EB2E3200BF
:10BF1000202020CEE1F0FBE2202020200020202065
:10BF20002020CAC7202020202000D0E5E6E8EC2011
:10BF3000E1F3E4E8EB00C2F0E5ECFF20E1F3E4E834
:10BF4000EB00C2F0E5ECFF2FC4E0F2E02000D3EFFD
:10BF5000F02E20F0E5EBE5202000202020CEE1F0BF
:10BF6000FBE220202000202020F1E2FFE7E8202053
:10BF7000200020202020CDE5F22020202000C2FB40
:10BF8000F5EEE420202020202000C2F0E5ECFF2088
:10BF9000202020202000C4E0F2E0202020202020CB
:10BFA0002000D3EFF02EE7F3ECECE5F02E00C1F328
:10BFB000E4E8EBFCEDE8EA203100C1F3E4E8EBFC57
:10BFC000EDE8EA203200C2FBF5EEE420202020005C
:10BFD0005520EFE8F22E203D2000CEE1F0FBE220DC
:10BFE000002020CAC7202000202D2D2D2D2000D17B
:10BFF000202000203E2000C12000323000520000EE
:020000040020DA
:08000000FFFFFFFFFFFFFFFF00
:020000040030CA
:0E000000FF080E1EFF8081FF0FC00FE00F40B3
:00000001FF
